:020000040000FA
:100000008E018F01900191019201013093009401C2
:1000100085018601980183168501803086000430B1
:1000200081008312861FDE2842208420980803194D
:100030001B28851598030B1D1B288B01B0200C086D
:10004000143A031D2528860185018C0B1B281428D2
:100050000F39820701340234043408341034203458
:10006000403400340034003400340F398207003447
:1000700000340034003400340034003401340234DD
:10008000043400346D308C008E0A0E08093C0318CD
:1000900008006F308C008E018F0A0F08053C031892
:1000A000080071308C008F01900A1008093C031879
:1000B000080073308C009001910A1108053C031868
:1000C000080072308C0091011308013C031872285B
:1000D000920A1208033C03187C286F308C009201AE
:1000E00093017C28920A1208093C03187C286E3080
:1000F0008C009201930A7C28120898009308031937
:1001000083280A30980708009501940A1408063CD1
:10011000031C94011408013A03199C28033A03199B
:10012000A128013A0319A428073A0319A728003087
:10013000860000308500080095151308031DA928C6
:10014000080015151208A92895141108A9281514D6
:100150001008970028208600170835208500080021
:10016000861B0800950803190800970A1708093C20
:10017000031C97011708A920D620861FBD28D6206A
:10018000861FBD2814309600861FB528D620960BF2
:10019000C428170894018F018E0195199300151931
:1001A0009200951891001518900014280C308C00BE
:1001B0000B1DD8288B018C0BD82808009601160837
:1001C000A920D620D620960A16080A3A031DDF2851
:0201D000DE2827
:02400E00F13F80
:00000001FF
